:020000001D29B8
:080008008C00030E8D00640062
:100010008E0A03198E039A0A0319990A0319980F75
:100020001828FC3098006C30990079309A009214AE
:100030009C0A03199B0F2128F0309B00BD309C00C7
:1000400092160D0E83008C0E0C0E0B110900820708
:10005000C134BE34BE34BE34C134FF34DE348034E7
:10006000FE34FF34DE34BC34BA34B634CE34BD345E
:10007000BE34AE349634B934F334EB34DB348034EC
:10008000FB348D34AE34AE34AE34B134E134D634D6
:10009000B634B634F934BF34B834B734AF349F34DF
:1000A000C934B634B634B634C934CF34B634B634C1
:1000B000B534C334FF34FF34C934FF34FF34073060
:1000C0009D00123095009601970193019401FC3038
:1000D00098006C30990079309A00F0309B00BD3068
:1000E0009C004030900000340030660017306500FE
:1000F00000340B118B178B1681016400D83062001D
:1001000081010034050812061039031900349206E3
:10011000121A00340E088F008E019401930110080A
:100120000F02031C9D28023C031C900A100891003A
:100130000310910C0310910C0034023E031C900339
:10014000003405301306FF300319C9280310140DBD
:100150008207150EBA281508BA280A30BA28160ED2
:10016000BA281608BA280A30BA28170EBA2817086B
:10017000BA2800340F399E009E079E079E079E07EF
:10018000031DC6289408FF300319C92813081E0749
:10019000272086001108D420930A06301306031D79
:1001A00000349301940A00349F009F0BD528080067
:1001B00005081D060739031900349D0664309E00AA
:1001C000FF30D4209E0BE0281D1D10299D1CEB281C
:1001D0001D1CF12800340A309E0010219E0BED28D2
:1001E0000034123015060319FC28073015070730B4
:1001F000831C013095070034013095000034921EB5
:1002000008299212073097070630831808299702A9
:10021000921C003492109701F0309B00BD309C007E
:100220000730160783181629960A003496006030A6
:100230001606031D00349601F1285F2074207920F2
:0A0240008220A120D820FF202029F1
:00000001FF
